:100000000C942A000C943F000C943F000C943F0089
:100010000C943F000C943F000C943F000C943F0064
:100020000C943F000C943F000C943F000C943F0054
:100030000C943F000C943F000C943F000C943F0044
:100040000C943F000C943F000C943F000C943F0034
:100050000C943F0011241FBECFE5D8E0DEBFCDBF1A
:1000600010E0A0E6B0E0E2E4F4E002C005900D92FA
:10007000AA38B107D9F70E945F000C941F020C94B4
:10008000000080E487B987E886B9089597B1907E2B
:1000900097B997B18770892B87B9369A349BFECF71
:1000A000349A24B135B1C901089520E040E050E010
:1000B000CA010197F1F72F5F2431D1F70895CF924C
:1000C000DF92EF92FF920F931F93CF93DF9380E025
:1000D00090E00197F1F783E00E94450181E060E044
:1000E0000E941D0180E487B987E886B980E690E028
:1000F0000E94760180E061E00E94EF018EE690E0D0
:100100000E94760120E040E050E0CA010197F1F73B
:100110002F5F2431D1F720E040E050E0CA01019781
:10012000F1F72F5F2431D1F720E040E050E0CA0121
:100130000197F1F72F5F2431D1F720E040E050E044
:10014000CA010197F1F72F5F2431D1F781E060E018
:100150000E941D018BE790E00E947601C0E0D0E094
:1001600087B1807E87B987B187B9369A349BFECF35
:10017000349AC4B0D5B087B1807E87B9389A369AA0
:10018000349BFECF349AE4B0F5B087B1807E87B956
:10019000399A369A349BFECF349A04B115B180E077
:1001A00061E00E94EF01C60164E070E00E948601F8
:1001B00085E061E00E94EF01C70164E070E00E9409
:1001C00086018AE061E00E94EF01C80164E070E00E
:1001D0000E94860120E0CE010197F1F72F5F2431C4
:1001E000D1F7BECF87B3807F87BB969A939882E082
:1001F0008A95F1F722E035E0C49A822F8A95F1F7CB
:1002000086B38295807F922F9A95F1F7C498932FA9
:100210009A95F1F7C49A922F9A95F1F796B3922F87
:100220009A95F1F7C498932F9A95F1F787FDE4CF4B
:10023000969887B38F6087BB0895282F662319F19E
:10024000939A82E08A95F1F7C49A88B3922F929597
:100250009F70807F982B98BB95E0892F8A95F1F746
:10026000C498892F8A95F1F7C49A88B32F70807F3C
:10027000822B88BB892F8A95F1F7C4989A95F1F75C
:100280000E94F20008959398DCCF1F93182F2CE260
:1002900031E040E951E0CA010197F1F721503040C7
:1002A000D1F787B38F6087BBBC9A8B9A8E9A88B33D
:1002B000807F88BBC4989698939881E08A95F1F7DF
:1002C000C49AC19A85E0982F9A95F1F7C4988A95B7
:1002D000F1F70E94F200812F8C6060E00E941D0106
:1002E00088E260E00E941D011F910895CF93DF9383
:1002F000EC018881882339F061E00E941D0121967C
:1003000088818823C9F7DF91CF910895EF92FF92FA
:100310000F931F93DF93CF9300D000D00F92CDB7F0
:10032000DEB79C018B017E010894E11CF11C85E085
:10033000F70111928A95E9F72115310591F0FE0137
:100340003596C9016AE070E00E94F8018083C90116
:100350006AE070E00E94F8019B0131976115710518
:1003600081F7FFEF0F3F1F0749F125E030E0201B29
:10037000310B25303105B4F4F701E20FF31F808112
:1003800089010F5F1F4FE00EF11E05C0F70181913B
:100390007F010F5F1F4F805D61E00E941D010530EE
:1003A0001105A4F30F900F900F900F900F90CF9125
:1003B000DF911F910F91FF90EF900895898188231D
:1003C00059F420E030E02F5F3F4FF701E20FF31FB9
:1003D00080818823C1F3CDCF20E030E0D1CF8832B7
:1003E00030F461118064806860E00E941D0108950E
:1003F00097FB092E07260AD077FD04D00CD006D033
:1004000000201AF4709561957F4F0895F6F7909546
:1004100081959F4F0895AA1BBB1B51E107C0AA1FDE
:10042000BB1FA617B70710F0A61BB70B881F991F95
:100430005A95A9F780959095BC01CD010895F8943F
:02044000FFCFEC
:1004420078426F6172642053656E736F72005465F7
:100452007374205574696C697479005323312020B8
:0A04620053233220205323332000DF
:00000001FF
